:100000000C9410050C9457050C9457050C94570547
:100010000C9457050C9457050C9457050C945705F0
:100020000C9457050C9457050C94640C0C94360DE5
:100030000C94331C0C9457050C9457050C945705DD
:100040000C9457050C9457050C9457050C945705C0
:100050000C9457050C94D31C0C9457050C9457051D
:100060000C9457050C9457050C9457050C945705A0
:100070000C9457050C9457050C9457050C94570590
:100080000C9457050C9457050C9457050C94570580
:100090000C9457050C9457050C9457050C94570570
:1000A0000C9457050C9457050C945705A30DC50DDA
:1000B000B30EC50DB30E0A0E2D0EB30E820E950EA5
:1000C000BB11BB11EA11EA1148128612A014A01448
:1000D0009F12A014A013A0137414A014A0148B14C6
:1000E0001F141A16041D1B062021150807091905DF
:1000F00022231C170A0B11801E352B39797A7B2C91
:100100002425180C0E0D1080742A31287C7D7E7FEA
:1001100026271213330F36802D2E302F3438378098
:100120004B6579626F6172642073746172742E0A18
:100130000055534220636F6E666967757265642E61
:100140000A000D0A696E69740A005B445D005B4336
:100150005D001203480048004B00420020006D0083
:100160006F00640000000E0374002E006D002E006E
:100170006B002E0000000403090409028D00050134
:1001800000A032090400000103010100092111014E
:1001900000012240000705810308000A090401004C
:1001A0000103010200092111010001224D00070590
:1001B000820308000A09040200010300000009216B
:1001C000110100012236000705830308000A090413
:1001D0000300020300000009211101000122220096
:1001E000070584032000010705040320000109041A
:1001F000040001030000000921110100012239005F
:10020000070585032000011201100100000008ED20
:10021000FEFECA04010102000105010906A1010553
:100220000719E029E71500250195087501810205E8
:10023000081901290595057501910295017503912C
:10024000010507190029F71500250195F8750181A9
:1002500002C00631FF0974A1010975150026FF00CF
:100260009520750881020976150026FF00952075F6
:10027000089102C005010980A101850216810026AE
:10028000B7001A81002AB700751095018100C005DA
:100290000C0901A1018503160100269C021A010028
:1002A0002A9C02751095018100C005010902A10177
:1002B0000901A10005091901290515002501950568
:1002C000750181029501750381010501093009312C
:1002D0001581257F95027508810609381581257FCE
:1002E000950175088106050C0A38021581257F9550
:1002F0000175088106C0C005010906A1010507199D
:10030000E029E71500250195087501810295017521
:1003100008810105081901290595057501910295C6
:1003200001750391010507190029FF150026FF003B
:10033000950675088100C0636F6E73756D65723ABE
:1003400020253034580A0073797374656D3A20257E
:100350003034580A000A002530325820006B657985
:10036000626F6172643A20004C45443A2025303275
:10037000580A00253032583A202530386225730A51
:1003800000722F632030313233343536370A00643F
:10039000656C5F6B65795F6269743A2063616E2793
:1003A000742064656C3A20253032580A0061646418
:1003B0005F6B65795F6269743A2063616E277420B0
:1003C0006164643A20253032580A004F6E657368C4
:1003D0006F743A2074696D656F75740A00290A009C
:1003E0002575002F002575005D280025640020007C
:1003F000256400200025640020002564007C002581
:10040000303258006D6F7573656B6579205B62746F
:100410006E7C782079207620685D287265702F6167
:10042000636C293A205B006D6B5F776865656C5F74
:1004300074696D655F746F5F6D6178203D20256420
:100440000A006D6B5F776865656C5F6D61785F73DF
:1004500070656564203D2025640A006D6B5F7469DA
:100460006D655F746F5F6D6178203D2025640A00C3
:100470006D6B5F6D61785F7370656564203D2025ED
:10048000640A006D6B5F696E74657276616C203D05
:100490002025640A006D6B5F64656C6179203D20E6
:1004A00025640A006D6B5F776865656C5F74696DC4
:1004B000655F746F5F6D6178203D2025640A006D73
:1004C0006B5F776865656C5F6D61785F737065659C
:1004D00064203D2025640A006D6B5F74696D655F63
:1004E000746F5F6D6178203D2025640A006D6B5F3D
:1004F0006D61785F7370656564203D2025640A0036
:100500006D6B5F696E74657276616C203D20256449
:100510000A006D6B5F64656C6179203D2025640A7B
:10052000000A00257500363A20776865656C5F74AF
:10053000696D655F746F5F6D61783A20000A002510
:100540007500353A20776865656C5F6D61785F731B
:10055000706565643A20000A00257500343A2074FD
:10056000696D655F746F5F6D61783A20000A0025E0
:100570007500333A206D61785F73706565643A2069
:10058000000A00257500323A20696E746572766142
:100590006C286D73293A20000A00257500313A2035
:1005A00064656C6179282A31306D73293A20000A1C
:1005B000092D2056616C756573202D0A004D3E0093
:1005C0004D25643E20003F007365742064656661BC
:1005D000756C740A00433E2000776865726520647C
:1005E000656C74613A20637572736F723D25642C7B
:1005F00020776865656C3D25640A536565206874DD
:1006000074703A2F2F656E2E77696B697065646917
:10061000612E6F72672F77696B692F4D6F757365E8
:100620005F6B6579730A000A092D204D6F7573653C
:100630006B6579202D0A4553432F713A097175690D
:10064000740A313A0964656C6179282A31306D7316
:10065000290A323A09696E74657276616C286D7385
:10066000290A333A096D61785F73706565640A34ED
:100670003A0974696D655F746F5F6D61780A353A28
:1006800009776865656C5F6D61785F737065656437
:100690000A363A09776865656C5F74696D655F74E1
:1006A0006F5F6D61780A0A703A097072696E742022
:1006B00076616C7565730A643A09736574206465C4
:1006C0006661756C74730A75703A092B310A646F30
:1006D000776E3A092D310A706775703A092B3130FF
:1006E0000A7067646F776E3A092D31300A0A7370A9
:1006F000656564203D2064656C7461202A206D610D
:10070000785F7370656564202A2028726570656162
:1007100074202F2074696D655F746F5F6D61782937
:100720000A003F004D3E2000433E20004C25640A55
:10073000000A092D20436F6E736F6C65202D0A45EA
:1007400053432F713A09717569740A6D3A096D6FD7
:100750007573656B65790A000A092D204D6167691B
:1007600063202D0A643A0964656275670A783A095C
:100770006465627567206D61747269780A6B3A0905
:100780006465627567206B6579626F6172640A6D7A
:100790003A096465627567206D6F7573650A763A0C
:1007A0000976657273696F6E0A733A0973746174BE
:1007B00075730A633A09636F6E736F6C65206D6FB2
:1007C00064650A302D343A096C61796572302D34D4
:1007D000284631302D4634290A506175733A096232
:1007E0006F6F746C6F616465720A6E3A094E4B529A
:1007F0004F0A003F004E4B524F3A206F66660A0088
:100800004E4B524F3A206F6E0A0074696D65725FED
:1008100072656164333228293A202530346C580AD5
:10082000006B6579626F6172645F6E6B726F3A2004
:1008300025580A006B6579626F6172645F69646C48
:10084000653A2025580A006B6579626F6172645FB2
:1008500070726F746F636F6C3A2025580A00686F6E
:1008600073745F6B6579626F6172645F6C656473EA
:1008700028293A2025580A000A092D20537461744A
:100880007573202D0A004743433A20342E392E3207
:10089000204156522D4C4942433A20312E382E30B9
:1008A00073766E204156525F415243483A2061763A
:1008B00072350A004F5054494F4E533A204C55461A
:1008C00041204D4F5553454B4559204558545241B1
:1008D0004B455920434F4E534F4C4520434F4D4DB0
:1008E000414E44204E4B524F204B45594D41505F95
:1008F00053454354494F4E20343039360A0042554F
:10090000494C443A20343139303537312D646972DD
:100910007479202830373A35353A3339204F6374AB
:100920002032382032303137290A005649443A20E3
:1009300030784645454428742E6D2E6B2E29205064
:1009400049443A203078434146452848484B4220A4
:100950006D6F6429205645523A203078303130345A
:100960000A00444553433A20742E6D2E6B2E206BA3
:100970006579626F617264206669726D7761726514
:1009800020666F722048484B42206D6F640A000A4F
:10099000092D2056657273696F6E202D0A000A6D4D
:1009A0006F7573653A206F66660A000A6D6F75731E
:1009B000653A206F6E0A000A6B6579626F61726436
:1009C0003A206F66660A000A6B6579626F6172642D
:1009D0003A206F6E0A000A6D61747269783A206F6E
:1009E00066660A000A6D61747269783A206F6E0A51
:1009F000000A64656275673A206F6E0A000A6465D2
:100A00006275673A206F66660A000A0A626F6F7441
:100A10006C6F616465722E2E2E2000433E20000014
:100A200011241FBECFEFDAE0DEBFCDBF04B603FE58
:100A300027C080914A0290914B02A0914C02B09144
:100A40004D028730904BA740B04BD1F410924A0230
:100A500010924B0210924C0210924D0214BE84B7B9
:100A6000877F84BF0FB6F894A89580916000886155
:100A700080936000109260000FBEE0E0F8E30995FB
:100A800011E0A0E0B1E0ECEBFAE402C005900D92B9
:100A9000A833B107D9F722E0A8E3B1E001C01D9265
:100AA000AA34B207E1F70E9492090C945C250C94D9
:100AB0000000FF93EF93E0913801F09139013097F6
:100AC00009F00995EF91FF910895FC01859180301F
:100AD00011F0EFDFFBCF0895FF27E0E230E247FFA0
:100AE0000CC0419597FF09C0EDE260957095809527
:100AF0009095611D711D811D911D27FF02C02195DB
:100B000030E350E2AA27660F771F881F991FAA1F9C
:100B1000A41710F0A41B63955A95A9F7AA3008F002
:100B2000A95FA05DAF93F3956115710581059105EE
:100B300041F7ED3211F4EF93F395F21718F43F9368
:100B4000F395FBCF8F91B5DFFA95E1F70895E99121
:100B5000F9918591803021F0853219F0AADFF9CF23
:100B6000089520E0E89455915532C1F3503311F4C3
:100B7000689455915A3348F4505390F3220F022E43
:100B8000220F220F200D250FF4CF0EF4219589910D
:100B90009991533619F3533729F1533559F1BC0163
:100BA00088279927E8945C3621F489919991689473
:100BB0005591543639F446EF7EF077FF0DC08FEF34
:100BC0009FEF0AC055374AE039F0583540E121F02F
:100BD000523642E009F00895FF93EF937DDFEF91E5
:100BE000FF91B7CFFF93EF93FC0181918030B9F370
:100BF00060DFFBCFFF93EF9368DFF1CFDF93CF93FD
:100C0000CDB7DEB72596A3DFCF91DF9108958FEFA3
:100C100084B980E485B957985F9A87B18F7387B993
:100C200088B1806C88B92E9A2F98E2E4F1E088E0D0
:100C30008E0F11928E13FDCFEAE3F1E088E08E0F64
:100C400011928E13FDCF82E491E090934D01809339
:100C50004C018AE391E090934B0180934A010895FF
:100C60000F931F93CF93DF9380914A0190914B0193
:100C700020914C0130914D0130934B0120934A015A
:100C800090934D0180934C01C0E0D0E001E010E072
:100C900080E090E025B1207C2C2BAC0133E0440FA8
:100CA000551F3A95E1F7242B25B9EAE1EA95F1F7CA
:100CB00000C0E0914A01F0914B01EC0FFD1F208133
:100CC00030E0082E02C0359527950A94E2F720FD02
:100CD0002F9AF5E3FA95F1F70000E6B52E982AE190
:100CE0002A95F1F700C040914C0150914D01DA0175
:100CF000AC0FBD1F4F9B0AC09801082E01C0220FE8
:100D00000A94EAF720953C91232308C06C9198013E
:100D1000082E01C0220F0A94EAF7262B2C9326B541
:100D20006E2F70E02E1718F026B530E004C026B5FF
:100D300030E021503F4F261B370B2630310558F04D
:100D4000E0914A01F0914B01EC0FFD1F2081FA0167
:100D5000EC0FFD1F20833AE13A95F1F700C02F9880
:100D60002E9AEBE2F1E03197F1F700C00000019616
:100D70008830910509F08ECFA0914C01B0914D01C2
:100D8000AC0FBD1FE0914A01F0914B01EC0FFD1F2C
:100D90009C918081981751F00E94711C60934E01C4
:100DA00070934F0180935001909351012196C83068
:100DB000D10509F06DCF80914102853021F08091FD
:100DC0004102811111C060914E0170914F018091DB
:100DD0005001909151010E94A71C61317742810519
:100DE000910510F00E94F21B81E0DF91CF911F91DD
:100DF0000F91089520914C0130914D01F901E80FB8
:100E0000F11D8081089508950895569A81FF02C0CA
:100E10005E9A08955E9808958091760108959FB72F
:100E2000F894109255019FBF90914102943009F0BF
:100E300057C09091E9009F703091EC00232F2170F2
:100E400030FD20E8922B24E02093E9002091EB0074
:100E500020FF43C02091EE0027FF3FC020915201A8
:100E6000222321F02091E80025FF37C01092520183
:100E700026E03091E80035FD15C030914102343054
:100E800061F53091EB0035FD28C0215021F481E05F
:100E90008093520122C0EFE9FFE03197F1F700C0E3
:100EA0000000E7CF8093F1008091E80085FD0AC043
:100EB0008091E80080FFFCCF8091E8008E778093DE
:100EC000E80006C08FB7F89421E0209355018FBF4A
:100ED0009F709093E90080E008959F709093E900DF
:100EE0008FEF0895CF93DF9300D01F92CDB7DEB779
:100EF0009C0180914102843019F593E099833B83F2
:100F00002A839093E9008FEF9091E800815095FD3E
:100F100006C095ED9A95F1F700008111F5CF80910B
:100F2000E80085FF0DC040E050E063E070E0CE01D6
:100F300001960E94540A8091E8008E778093E80021
:100F40000F900F900F90DF91CF910895CF93DF9383
:100F500000D01F92CDB7DEB720914102243021F599
:100F600022E029839B838A8383E08093E9008FEFCB
:100F70009091E800815095FD06C095ED9A95F1F7A6
:100F800000008111F5CF8091E80085FF0DC040E0A1
:100F900050E063E070E0CE0101960E94540A809117
:100FA000E8008E778093E8000F900F900F90DF910C
:100FB000CF910895209141022430F1F422E0209352
:100FC000E9002FEF3091E800215035FD06C035EDE6
:100FD0003A95F1F700002111F5CF2091E80025FFA7
:100FE0000BC040E050E065E070E00E94540A809140
:100FF000E8008E778093E8000895CF93DF932091E7
:101000004102243009F048C0EC0180910A01882394
:10101000E1F080910B018823C1F085E08093E90025
:101020008FEF9091E800815095FD06C09AE29A9565
:10103000F1F700C08111F5CF8091E80085FF2CC049
:1010400040E050E060E270E017C081E08093E9008A
:101050008FEF9091E800815095FD06C095ED9A952F
:10106000F1F700008111F5CF8091E80085FF14C0F1
:1010700040E050E068E070E0CE010E94540A8091A8
:10108000E8008E778093E80080E2FE01A6E5B1E0FB
:1010900001900D928A95E1F7DF91CF9108958EE44A
:1010A00091E00E94650580914002811109C00E9473
:1010B000E90B0E94460C8091E20084608093E2007C
:1010C00008958AE491E00E94650510924002089517
:1010D0000895209153012F5F822F62E30E94222501
:1010E000992319F020935301089510925301809190
:1010F0005501882371F180914102843041F580913E
:10110000E9008F702091EC00922F917020FD90E803
:10111000892B94E09093E9009091EB0090FF14C02C
:101120009091EE0097FF10C09091E80095FF03C0EA
:101130001092F100F9CF9091E80090FF05C09091D6
:10114000E8009E779093E8008F708093E9001092FA
:101150005501089542E061EC81E00E94630B42E09A
:1011600061EC82E00E94630B42E061EC83E00E944C
:10117000630B42E261EC84E00E94630B42E261ECAB
:1011800085E00C94630B80914302833009F455C0D1
:1011900030F4813071F0823009F48EC008958A30C5
:1011A00009F47AC08B3009F460C0893009F09CC022
:1011B00020C080914202813A09F096C08091E800F7
:1011C000877F8093E8008091460290914702892BA7
:1011D00021F460E286E591E003C060E080E090E009
:1011E00070E00E949F0A8091E8008B778093E8006E
:1011F000089580914202813209F076C080914602C2
:1012000090914702009719F0049709F06DC0809102
:10121000E800877F8093E8008091E80082FD05C0A8
:10122000809141028111F8CF5FC08091F1008093DD
:1012300076018091E8008B7753C080914202813A19
:1012400009F052C08091460290914702892B09F023
:101250004BC08091E800877F8093E8008091E80090
:1012600080FFFCCF80910A0136C08091420281321A
:10127000D9F58091460290914702892BA9F580917A
:10128000E800877F8093E8000E94980B80914402D9
:1012900080930A010C94C21480914202813221F59C
:1012A0008091E800877F8093E8000E94980B8091EE
:1012B000450280937701089580914202813AA1F41A
:1012C0008091E800877F8093E8008091E80080FFAC
:1012D000FCCF809177018093F1008091E8008E77B8
:1012E0008093E8000C94980B0895089508958091D8
:1012F0007601809354011092760180E00E940507E8
:101300000E945F100C94C2140C9477090E94F21B87
:1013100080913F02882329F00E941B1C81110C94AC
:101320003E0A089584B7877F84BF0FB6F894A895C6
:1013300080916000886180936000109260000FBE11
:1013400090E080E80FB6F89480936100909361007C
:101350000FBE8FE097E00E94C31B82E491E00E94E1
:1013600065050E9475090E948C0F0E94E90B0E947E
:10137000460C8091E20084608093E2007894809132
:1013800041028430E1F781E391E00E9465050E940B
:101390008E0F80E091E00E94CB0E80E291E00E94EF
:1013A00065050E94760980914102853019F40E94FA
:1013B0008609F9CF0E94920FF6CF0E942F1C8091D0
:1013C00054018093760108950C94DD09292F332769
:1013D00023303105C9F064F42130310581F0223029
:1013E000310509F043C08DE890E02AE731E042C0C2
:1013F00021323105F1F02232310541F137C082E16D
:1014000090E027E032E036C099278130910541F025
:101410008230910541F0892B49F5E6E7F1E005C0FE
:10142000E6E6F1E002C0E2E5F1E0849190E09F01A0
:1014300021C06530D8F4E62FF0E0EE0FFF1FED5D20
:10144000FE4F2081318189E090E014C0653070F456
:1014500070E0FB01EE0FFF1FE75EFE4F2081318140
:10146000FB01EC5EFE4F808190E004C080E090E0E4
:1014700020E030E0FA0131832083089580E189BDC6
:1014800082E189BD09B400FEFDCF8091D8008F7D37
:101490008093D8008091E00082608093E00080918A
:1014A000E00081FDFCCF0895CF92DF92EF92FF9292
:1014B0000F931F93CF93DF93EC018B016A010E947E
:1014C000B70B811133C0C114D10439F0F60180810A
:1014D0009181081B190BC80FD91FE12CF12C0115A4
:1014E000110519F18091E80085FD16C08091E80092
:1014F0008E778093E800C114D10449F0F601808111
:101500009181E80EF91EF182E08285E00FC00E9411
:10151000B70B882321F30AC089918093F100015011
:101520001109FFEFEF1AFF0ADACF80E0DF91CF91C8
:101530001F910F91FF90EF90DF90CF900895209131
:101540004802309149022617370748F061157105A6
:1015500039F42091E8002E772093E80001C0B9010A
:1015600040E061157105A9F120914102222309F49F
:1015700043C0253009F442C02091E80023FD40C05B
:101580002091E80022FD32C02091E80020FFE9CF41
:101590004091F3002091F20030E0342BFC01CF01A8
:1015A0006115710559F02830310540F4819180931F
:1015B000F100615071092F5F3F4FF1CF41E02830BA
:1015C000310509F040E02091E8002E772093E800F3
:1015D000C8CF4111C9CF0AC080914102882361F070
:1015E000853061F08091E80083FD0AC08091E800B9
:1015F00082FFF2CF80E0089582E0089583E00895AD
:1016000081E008952091480230914902261737075A
:1016100048F06115710539F42091E8002E77209388
:10162000E80001C0B901FC0120E06115710591F1EC
:1016300080914102882309F440C0853009F43FC0FD
:101640008091E80083FD3DC08091E80082FD2FC0BD
:101650008091E80080FFE9CF2091F3008091F200B3
:1016600090E0922B6115710559F08830910540F496
:1016700024912093F1003196615071090196F2CFC7
:1016800021E0089709F020E08091E8008E778093B0
:10169000E800CBCF2111CCCF0AC080914102882332
:1016A00061F0853061F08091E80083FD0AC080918F
:1016B000E80082FFF2CF80E0089582E0089583E0A1
:1016C000089581E00895982F973058F59093E90098
:1016D000981739F07091EC002091ED005091F000D6
:1016E00003C0242F762F50E021FF19C03091EB006A
:1016F0003E7F3093EB003091ED003D7F3093ED0065
:101700003091EB0031603093EB007093EC0020934C
:10171000ED005093F0002091EE0027FF07C09F5F7F
:10172000D3CF8F708093E90081E0089580E0089521
:101730008091420287FF11C08091E80082FD05C0C0
:10174000809141028111F8CF11C08091E8008B7720
:101750000BC080914102882349F08091E80080FF0E
:10176000F8CF8091E8008E778093E800089520916B
:10177000E4003091E50095E64091EC00842F817003
:1017800040FF22C08091E80080FD1CC08091410292
:10179000882391F0853091F08091EB0085FD10C099
:1017A0004091E4005091E5004217530729F39A0154
:1017B000915011F784E0089582E0089583E0089540
:1017C00081E0089580E008954091E80042FFDECF77
:1017D00008950E94570C0E945F0CE0EEF0E08081BB
:1017E00081608083E8EDF0E080818F77808319BC91
:1017F000A7EDB0E08C918E7F8C9380818F7E80836B
:101800001092400208950F931F93CF93DF930E948D
:10181000570C0E945F0CC8EDD0E088818F778883D9
:1018200088818068888388818F7D888319BC109225
:10183000410210923D0210923F0210923E0200EED1
:1018400010E0F80180818B7F8083888181608883AC
:1018500042E060E080E00E94630BE1EEF0E0808116
:101860008E7F8083E2EEF0E08081816080838081E2
:1018700088608083F80180818E7F80838881806189
:101880008883DF91CF911F910F910895E8EDF0E0EB
:1018900080818F7E8083E7EDF0E0808181608083AE
:1018A00084E082BF81E0809340020C94030CE8ED59
:1018B000F0E080818E7F80831092E2000895109284
:1018C000DA001092E10008951F920F920FB60F9266
:1018D00011242F933F934F935F936F937F938F9335
:1018E0009F93AF93BF93EF93FF938091E10082FFAB
:1018F0000BC08091E20082FF07C08091E1008B7FE6
:101900008093E1000E9469088091DA0080FF1FC087
:101910008091D80080FF1BC08091DA008E7F809379
:10192000DA008091D90080FF0DC080E189BD82E19D
:1019300089BD09B400FEFDCF81E0809341020E9481
:101940004F0805C019BC109241020E9461088091A5
:10195000E10080FF19C08091E20080FF15C08091F6
:10196000E2008E7F8093E2008091E20080618093AC
:10197000E2008091D80080628093D80019BC85E095
:10198000809341020E9484098091E10084FF30C06D
:101990008091E20084FF2CC080E189BD82E189BD95
:1019A00009B400FEFDCF8091D8008F7D8093D800D0
:1019B0008091E1008F7E8093E1008091E2008F7E34
:1019C0008093E2008091E20081608093E200809148
:1019D0003D02882311F084E007C08091E30087FD79
:1019E00002C081E001C083E0809341020E94E409CB
:1019F0008091E10083FF29C08091E20083FF25C030
:101A00008091E100877F8093E10082E08093410232
:101A100010923D028091E1008E7F8093E1008091E1
:101A2000E2008E7F8093E2008091E20080618093EB
:101A3000E20042E060E080E00E94630B8091F000F1
:101A400088608093F0000E946808FF91EF91BF9139
:101A5000AF919F918F917F916F915F914F913F9146
:101A60002F910F900FBE0F901F9018951F920F92FD
:101A70000FB60F9211242F933F934F935F936F9361
:101A80007F938F939F93AF93BF93CF93DF93EF9306
:101A9000FF93C091E900CF708091EC00D82FD170F6
:101AA00080FDD0E81092E9008091F000877F80935C
:101AB000F00078940E947A0D1092E9008091F00075
:101AC00088608093F000CD2BCF70C093E900FF9128
:101AD000EF91DF91CF91BF91AF919F918F917F91C6
:101AE0006F915F914F913F912F910F900FBE0F908B
:101AF0001F9018951F93CF93DF93CDB7DEB7AA97AA
:101B00000FB6F894DEBF0FBECDBFE2E4F2E088E08E
:101B10008E0F9091F10091938E13FBCF0E94C3081A
:101B20008091E80083FF1FC180914202909143029F
:101B3000492F50E04A30510508F015C1FA01EA5A20
:101B4000FF4F0C944225803881F0823809F00BC198
:101B5000809146028F708093E9008091EB0085FBB5
:101B6000882780F91092E90006C080913E0290918A
:101B70003F02911182609091E800977F9093E80076
:101B80008093F1001092F100C8C0282F2D7F09F03A
:101B9000EAC0882319F0823061F0E5C080914402E8
:101BA000813009F0E0C0933009F080E080933F027B
:101BB0002BC080914402811127C0809146028F7012
:101BC00009F4D1C08093E9002091EB0020FF1CC0F4
:101BD000933021F48091EB00806214C09091EB006F
:101BE00090619093EB0021E030E0A90102C0440F26
:101BF000551F8A95E2F74093EA001092EA0080911F
:101C0000EB0088608093EB001092E9008091E8007F
:101C1000877F86C08111A7C0109144021F778091F1
:101C2000E3008078812B8093E3008091E800877F38
:101C30008093E8000E94980B8091E80080FFFCCF21
:101C40008091E30080688093E300111102C082E07C
:101C500001C083E08093410286C08058823008F042
:101C600082C080914402909145028C3D53E09507DB
:101C700079F583E08A838AE289834FB7F894DE019D
:101C8000139620E03EE051E2E32FF0E0509357003E
:101C9000E49120FF03C0E295EF703F5FEF708E2F5D
:101CA00090E0EA3010F0C79601C0C0968D939D93E6
:101CB0002F5F243149F74FBF8091E800877F8093E1
:101CC000E8006AE270E0CE0101960E949F0A14C00B
:101CD000AE014F5F5F4F609146020E94E609BC0172
:101CE000892B09F440C09091E800977F9093E80019
:101CF00089819A810E94020B8091E8008B77809302
:101D0000E80031C0803879F58091E800877F8093C2
:101D1000E80080913D028093F1008091E8008E7789
:101D20008093E8000E94980B1EC081111CC0909106
:101D300044029230C0F48091E800877F8093E800ED
:101D400090933D020E94980B80913D02811106C044
:101D50008091E30087FD02C081E001C084E08093B0
:101D600041020E94AA088091E80083FF0AC0809186
:101D7000E800877F8093E8008091EB008062809389
:101D8000EB00AA960FB6F894DEBF0FBECDBFDF9171
:101D9000CF911F91089590937D0180937C010895C8
:101DA000E0917C01F0917D01309721F00190F0816C
:101DB000E02D099480E00895EF92FF920F931F9316
:101DC000CF93DF93E0917C01F0917D013097B1F1E9
:101DD0008C010280F381E02D099580912C0282FF15
:101DE0002DC080FF04C08DE593E00E946505E801E9
:101DF00010E287E5E82E83E0F82E80912C0280FF28
:101E00000BC088811F928F93FF92EF920E94FE0574
:101E10000F900F900F900F90115021961111EDCF50
:101E200080912C0280FF0AC085E593E0DF91CF917D
:101E30001F910F91FF90EF900C946505DF91CF916A
:101E40001F910F91FF90EF900895E0917C01F09128
:101E50007D01309721F00480F581E02D09940895EB
:101E6000CF93DF93EC0180917A0190917B01C817A9
:101E7000D90709F1D0937B01C0937A01E0917C01ED
:101E8000F0917D013097B9F00680F781E02DCE0109
:101E9000099580912C0282FF0EC080FF0CC0DF9359
:101EA000CF9387E493E09F938F930E94FE050F905A
:101EB0000F900F900F90DF91CF910895CF93DF9304
:101EC000EC018091780190917901C817D90709F147
:101ED000D0937901C0937801E0917C01F0917D016C
:101EE0003097B9F00084F185E02DCE0109958091FD
:101EF0002C0282FF0EC080FF0CC0DF93CF9387E3DC
:101F000093E09F938F930E94FE050F900F900F9088
:101F10000F90DF91CF9108950C9460100E945C1C8B
:101F20000C9407065F926F927F928F929F92AF926E
:101F3000BF92CF92DF92EF92FF920F931F93CF93B6
:101F4000DF9300D000D01F92CDB7DEB70E943006DD
:101F50008FE7C82E81E0D82E512C88248394912CB1
:101F6000852D0E94FA06A82EF601E080E82641F4AD
:101F70005394FFEFCF1ADF0A88E05812F1CF40C028
:101F800080912C0281FD0E94611000E010E0F12C94
:101F9000B12CC701002E02C0959587950A94E2F7EF
:101FA00080FF28C009835A823401002E02C0660CCB
:101FB000771C0A94E2F793012A213B2181E0232B2D
:101FC00009F480E08B830E94651C8160782F9D83DB
:101FD0008C8349815A816B818D810E949510498142
:101FE0005A816B817C818D810E94DF1BF60180818B
:101FF000682660820F5F1F4F0830110551F6B8CF79
:102000008FEF89838A831B820E94651C8160782FF1
:102010009D838C8349815A816B818D810E949510AB
:102020000E94DE1B0E94521F10917E010E94D00E62
:10203000181771F10E94D00E80937E0190912C02AE
:1020400092FF0EC090FF0CC01F928F9388E693E022
:102050009F938F930E94FE050F900F900F900F900B
:1020600080917E010F900F900F900F900F90DF9155
:10207000CF911F910F91FF90EF90DF90CF90BF9085
:10208000AF909F908F907F906F905F900C94F01B1B
:102090000F900F900F900F900F90DF91CF911F91A5
:1020A0000F91FF90EF90DF90CF90BF90AF909F90F7
:1020B0008F907F906F905F9008950C94050708951E
:1020C0000895EF92FF920F931F93CF93DF9381E8D0
:1020D00093E00E946505C0E0D0E08DE2E82E81E04B
:1020E000F82E03E713E08C2F0E94FA060E94C81B0B
:1020F000FF92EF921F928F93DF93CF931F930F93D3
:102100000E94FE0521968DB79EB708960FB6F894EB
:102110009EBF0FBE8DBFC830D10529F7DF91CF918B
:102120001F910F91FF90EF900895CF93DF93CDB75C
:10213000DEB72B970FB6F894DEBF0FBECDBF942F3E
:102140004F83252F588769877A878B874A855B85D8
:10215000452B21F02F3F09F59F3FF9F4DE01119641
:1021600086E0FD0111928A95E9F785E0FE01379638
:1021700001900D928A95E1F749815A816B817C81AA
:102180008D819E810E94A7172B960FB6F894DEBF13
:102190000FBECDBFDF91CF9108954F8158856985DE
:1021A0007A858B850E94DF1BD9CFCF93882309F4D2
:1021B00065C0C82F8CEF8C0F813A20F080E58C0F22
:1021C0008E3248F48C2F0E949C22811157C08C2F94
:1021D0000E947F1A0CC080E28C0F883058F4C770C0
:1021E00081E001C0880FCA95EAF70E942A1BCF91AF
:1021F0000C946E1B8BE58C0F833078F4C53A29F074
:10220000C63A31F083E890E005C081E890E002C072
:1022100082E890E0CF910C94300F88E58C0F8531E7
:1022200068F5C83A89F0C93A91F0CA3A99F0CB3AC0
:10223000A1F0CC3AA9F0CD3AB1F0CE3AB9F0CF3A0C
:10224000C1F080E090E017C082EE90E014C089EE0B
:1022500090E011C08AEE90E00EC085EB90E00BC0DC
:1022600086EB90E008C083EB90E005C084EB90E043
:1022700002C087EB90E0CF910C945E0FCF91089550
:10228000882349F19CEF980F913A20F090E5980F40
:102290009E3218F40E94D21A0DC090E2980F983026
:1022A00058F4877091E001C0990F8A95EAF7892F59
:1022B0000E94301B0C946E1B9BE5980F933020F40A
:1022C00080E090E00C94300F885A853120F480E053
:1022D00090E00C945E0F0895882321F00E942A1B41
:1022E0000C946E1B0895882321F00E94301B0C94DF
:1022F0006E1B0895BF92CF92DF92EF92FF920F93E1
:102300001F93CF93DF9300D000D000D0CDB7DEB7BE
:1023100025E0FC01DE01119601900D922A95E1F76E
:10232000FC01408151810281638174812581229564
:102330002F706115710509F403C35F3F19F44F3F16
:1023400009F4FEC26C01862F7D836C83602F782F89
:102350008D812E830E94031A182FB92E0E94021A13
:102360000E94F218EB2DE295EF70F0E0E05AFF4F7B
:102370002E810C9442258B2D807F9B2D9F70F92EF2
:10238000882319F0F29490EFF922002349F0FF20FE
:1023900009F483C28F2D0E943D1B0E946E1B7DC2DB
:1023A000812F0E944011FF2009F4CAC28F2D0E9484
:1023B000431B26960FB6F894DEBF0FBECDBFDF914C
:1023C000CF911F910F91FF90EF90DF90CF90BF9032
:1023D0000C946E1B8B2D807F9B2D9F70F92E80326D
:1023E00019F0F29480EFF822112319F0113009F15D
:1023F0002AC00023B1F08F2D222351F1213041F565
:1024000026960FB6F894DEBF0FBECDBFDF91CF91F9
:102410001F910F91FF90EF90DF90CF90BF900C94A1
:102420004D1B222319F0213009F48AC20E94561B49
:102430002DC00023F1F0263008F082C20E94271B35
:102440008F2129F023C00023F9F0211116C08F2D10
:1024500026960FB6F894DEBF0FBECDBFDF91CF91A9
:102460001F910F91FF90EF90DF90CF90BF900C9451
:102470006C11253008F064C209C0F601858180FF27
:102480000CC28F708583E3CF21111CC28F2D83C1B5
:102490002B2D26952695237030E02115310521F04E
:1024A00021303105D1F04CC2002321F0812F9B2D2A
:1024B000937002C080E090E026960FB6F894DEBFDD
:1024C0000FBECDBFDF91CF911F910F91FF90EF9085
:1024D000DF90CF90BF900C94300F002321F0812F1C
:1024E0009B2D937002C080E090E026960FB6F89482
:1024F000DEBF0FBECDBFDF91CF911F910F91FF9037
:10250000EF90DF90CF90BF900C945E0F812F00234F
:1025100019F00E94D81D02C00E94401E26960FB6D8
:10252000F894DEBF0FBECDBFDF91CF911F910F9109
:10253000FF90EF90DF90CF90BF900C94C51E8B2D35
:10254000837009F07BC00111FBC1812F82958695B4
:102550008770880F880F912F9F70C92ED12CE12C86
:10256000F12C082E04C0CC0CDD1CEE1CFF1C0A94C0
:10257000D2F714FF12C04FE050E060E070E004C0FA
:10258000440F551F661F771F8A95D2F7CB01BA01FA
:10259000609570958095909503C060E070E0CB01E8
:1025A0002B2D269526952370422F50E04230510561
:1025B000D9F04330510569F16C297D298E299F2975
:1025C0004130510551F126960FB6F894DEBF0FBE8B
:1025D000CDBFDF91CF911F910F91FF90EF90DF90D2
:1025E000CF90BF900C9417196C297D298E299F29B3
:1025F00026960FB6F894DEBF0FBECDBFDF91CF9108
:102600001F910F91FF90EF90DF90CF90BF900C94AF
:1026100031190E941719C701B60126960FB6F89412
:10262000DEBF0FBECDBFDF91CF911F910F91FF9005
:10263000EF90DF90CF90BF900C94FD18002319F01D
:102640008B2D817001C08695882309F479C1812F73
:10265000829586958770880F880F912F9F70C92E5D
:10266000D12CE12CF12C082E04C0CC0CDD1CEE1C6E
:10267000FF1C0A94D2F714FF12C04FE050E060E054
:1026800070E004C0440F551F661F771F8A95D2F76C
:10269000CB01BA01609570958095909503C060E07C
:1026A00070E0CB012B2D269526952370422F50E00C
:1026B00042305105D9F04330510569F16C297D292B
:1026C0008E299F294130510551F126960FB6F89475
:1026D000DEBF0FBECDBFDF91CF911F910F91FF9055
:1026E000EF90DF90CF90BF900C94DE196C297D297C
:1026F0008E299F2926960FB6F894DEBF0FBECDBF58
:10270000DF91CF911F910F91FF90EF90DF90CF90CD
:10271000BF900C94F0190E94DE19C701B6012696ED
:102720000FB6F894DEBF0FBECDBFDF91CF911F91E2
:102730000F91FF90EF90DF90CF90BF900C94CC1949
:10274000103FD1F128F480E4810F803250F0A0C016
:10275000123F09F462C008F44BC0133F09F472C081
:1027600097C0F12FF071FF2E8B2D8F71002351F048
:102770000E946519812FFF2019F08295807F68CE15
:102780008F7066CE0E948619812FFF2019F08295E6
:10279000807F01C08F7026960FB6F894DEBF0FBE03
:1027A000CDBFDF91CF911F910F91FF90EF90DF9000
:1027B000CF90BF900C9473110023B1F0253008F036
:1027C000BFC08B2D8F7126960FB6F894DEBF0FBE5B
:1027D000CDBFDF91CF911F910F91FF90EF90DF90D0
:1027E000CF90BF900C94AB19263008F0A9C0E9CF68
:1027F0000023A9F08B2D8F7126960FB6F894DEBFBB
:102800000FBECDBFDF91CF911F910F91FF90EF9041
:10281000DF90CF90BF900C946519002359F38B2D56
:102820008F7126960FB6F894DEBF0FBECDBFDF9135
:10283000CF911F910F91FF90EF90DF90CF90BF90BD
:102840000C948619002399F08B2D8F7126960FB664
:10285000F894DEBF0FBECDBFDF91CF911F910F91D6
:10286000FF90EF90DF90CF90BF900C945019269678
:102870000FB6F894DEBF0FBECDBFDF91CF911F9191
:102880000F91FF90EF90DF90CF90BF900C944B1979
:102890000023A9F0222309F4ADCF812F26960FB68D
:1028A000F894DEBF0FBECDBFDF91CF911F910F9186
:1028B000FF90EF90DF90CF90BF900C94D510222323
:1028C00009F4ADCF812F26960FB6F894DEBF0FBE68
:1028D000CDBFDF91CF911F910F91FF90EF90DF90CF
:1028E000CF90BF900C9440114B2D4F70612FC601BB
:1028F0000E94521D26960FB6F894DEBF0FBECDBFC4
:10290000DF91CF911F910F91FF90EF90DF90CF90CB
:10291000BF900C944B184B2D4F70612FC60126961B
:102920000FB6F894DEBF0FBECDBFDF91CF911F91E0
:102930000F91FF90EF90DF90CF90BF900C94551DBA
:1029400026960FB6F894DEBF0FBECDBFDF91CF91B4
:102950001F910F91FF90EF90DF90CF90BF9008955F
:102960000E944A1B0E94191B0E946E1B0E94F71FA7
:102970000E94C51E80E090E00E94300F80E090E051
:102980000C945E0F0E943A1B0C94B014CF93DF930B
:1029900000D000D01F92CDB7DEB7942F4983252FEA
:1029A0005A836B837C838D834C815D81452B39F108
:1029B0002F3F11F49F3F19F149815A816B817C812E
:1029C0008D810E94031A292F22952F7030E02C3020
:1029D000310504F52A3031055CF4225031092230EA
:1029E000310568F4853A80F4843090F4823080F0C8
:1029F000883E38F4803E60F48450813A48F080E0AC
:102A000014C0803FE1F704C090E2980F983080F73F
:102A100081E00BC02C30310521F493FB882780F92D
:102A200004C02F303105C9F3EACF0F900F900F90FB
:102A30000F900F90DF91CF910895CF93DF9300D047
:102A400000D01F92CDB7DEB70F900F900F900F9070
:102A50000F90DF91CF910895CF93DF9300D000D0F6
:102A600000D0CDB7DEB726960FB6F894DEBF0FBE06
:102A7000CDBFDF91CF9108951F93CF93DF93C09186
:102A8000870116E080918801C81799F0D0E01C9F5B
:102A9000F0011D9FF00D1124E757FE4F4081518139
:102AA00062817381848195810E942C152196C77063
:102AB000E9CFDF91CF911F9108954091B9015091D5
:102AC000BA016091BB017091BC018091BD019091F0
:102AD000BE010C942C158091BE0182958F7009F077
:102AE00054C08091BB01882309F44FC080918701B5
:102AF000A09188016091B9017091BA014091BC0127
:102B00005091BD01B6E08A1709F43FC090E041152D
:102B10005105C1F17F3F11F46F3FA1F1B89FF00162
:102B2000B99FF00D1124E757FE4F218172132AC07F
:102B30002081621327C02281211124C02381348186
:102B40002417350710F421503109241B350B2C3282
:102B50003140C0F42091BE012F7020612093BE014E
:102B600026E0289FF001299FF00D1124E257FE4F27
:102B700080818F708061808389EB91E00E947A115F
:102B80000C943C1501968770BECF0895BF92CF92EA
:102B9000DF92EF92FF920F931F93CF93DF93CDB706
:102BA000DEB761970FB6F894DEBF0FBECDBF7C01D4
:102BB00085E0F701DE011D9601900D928A95E1F7FF
:102BC000D7014C9111965C9111971296DC90129757
:102BD00013960D911C9114973091B9016091BA012F
:102BE0008091BC019091BD01009709F47FC16F3FB6
:102BF00019F43F3F09F47AC1B090BB01BB2009F43E
:102C0000CAC02091BE010817190750F0F801E81B4F
:102C1000F90BCF01CC24C3948C329140D0F009C081
:102C200080959095800F911FCC24C3948C32914055
:102C300080F0C12C207F09F0CCC0702F198B088B3D
:102C40006D2D89890E941D1589EB91E00E947A11F2
:102C5000B6C0822F807F09F047C0651314C03413BB
:102C600012C0D11010C02F7020612093BE010E94AD
:102C70005D1589EB91E00E947A118091BE01D70128
:102C800015968C932FC00115110519F15F3F11F4B2
:102C90004F3FF9F0CD2CD1101CC0809187012091BD
:102CA000880136E0821709F45CC090E0389FF0019B
:102CB000399FF00D1124E757FE4F6181561306C06E
:102CC0006081461303C06281611103C00196877061
:102CD000E9CFCD2CDD2009F429C18091BE018160AE
:102CE0008093BE01C12C22C1651308C0341306C0F5
:102CF000D11004C08091BE01D701CCC04D875E8742
:102D0000DF86702F198B088B6D2D89890E94C61460
:102D10008823E9F1DD20D9F12091BE01822F82952F
:102D20008F7090E0029774F08091B9019091BA0190
:102D300098878F8319861B870A872C87CE01079671
:102D40000E947A1186E0F701A9EBB1E001900D92A3
:102D50008A95E1F70E946B150E945D15CC24C394FF
:102D6000E5C0702F198B088B60E089890E94031AD7
:102D7000292F22952F7030E0223031050CF0CAC087
:102D80009F7009F0C4C0805E883008F4CFC0C701CE
:102D90000E947A11E3CF0817190708F456C0F8010A
:102DA000E81BF90BCF018C32914008F456C0C12CBE
:102DB000702F198B088B6D2D89890E941D15E9EBE9
:102DC000F1E086E0DF011D928A95E9F70E945D152A
:102DD000ADC0651314C0341312C0D11010C080915F
:102DE000BE01F7018583C7010E947A1186E0E9EBF5
:102DF000F1E0DF011D928A95E9F7CB2C97C04D8752
:102E00005E87DF86702F198B088B6D2D89890E9454
:102E1000C614882309F4BBCFDD2009F4B8CF209174
:102E2000BE01822F82958F7090E002970CF48ACFBA
:102E30008091B9019091BA019A8389831B821D8385
:102E40000C832E83CE0101967BCF80959095800FC9
:102E5000911F8C32914008F0AACFCD2CDD2009F4CF
:102E600096CF65132EC034132CC02091BE0120FDD7
:102E70001FC0822F82958F70D9F0D70115962C93A1
:102E800015978F3049F08F5F982F9295907F822F02
:102E90008F70892B15968C93C7010E947A1186E05A
:102EA000F701A9EBB1E001900D928A95E1F78ECF81
:102EB00086E0F701A9EBB1E001900D928A95E1F768
:102EC00035C04D875E87DF86702F198B088B6D2D7F
:102ED00089890E94C614811135CF8091BE0181601D
:102EE0008093BE01C7010E947A1120C0DD2009F441
:102EF0004ECF4D875E87DF86702F198B088B6D2D27
:102F000089890E94C614882309F441CF1BCF8111FF
:102F10003ACF0CC0243031050CF039CF9F7009F442
:102F200032CFF7019581907F09F02DCF8C2D6196DE
:102F30000FB6F894DEBF0FBECDBFDF91CF911F91CA
:102F40000F91FF90EF90DF90CF90BF9008951F9367
:102F5000CF93DF93CDB7DEB72C970FB6F894DEBFD3
:102F60000FBECDBF4F83588769877A878B879C8731
:102F7000CE0107960E94C615882369F08F81988537
:102F80002A853B85232BF1F19F3F09F063C08F3FDA
:102F900009F060C037C086E0FE013796DE01119669
:102FA00001900D928A95E1F76F817885EA85FB851E
:102FB000309741F17F3F11F46F3F21F1209188015B
:102FC00030E0C9010196877099274091870150E050
:102FD0008417950709F447C069837A83FD83EC83DE
:102FE00096E0929FD001939FB00D1124A757BE4F3A
:102FF000FE01319601900D929A95E1F78093880138
:103000000E943C1516E080918701909188018917F4
:10301000C1F1189FC001112487579E4F0E94C61509
:10302000882379F1E09187011E9FF0011124E75771
:10303000FE4F4081518162817381848195810E941C
:103040002C158091870190E00196877099278093D5
:103050008701D9CF4F81588569857A858B859C8575
:103060000E942C15CFCF0E94C2141092880110929A
:103070008701E9EBF1E086E0DF011D928A95E9F72F
:10308000C1CF2C960FB6F894DEBF0FBECDBFDF9137
:10309000CF911F910895DF92EF92FF920F931F93AC
:1030A000CF93DF93FC01892B09F48AC0E12CF12C2A
:1030B000DD24D394EF0121968491853709F461C012
:1030C00058F4843708F04EC0843008F06AC081306C
:1030D000D1F0823071F174C0883709F45DC050F4CA
:1030E000863709F455C0873709F06AC08E2D0E94D3
:1030F000371B54C09CE7980F903708F061C08F775A
:103100000E94401150C08F010E5F1F4FFE0184913D
:1031100090E2980F983050F48770FD2D01C0FF0F9A
:103120008A95EAF78F2F0E943D1B14C00E94D5108C
:1031300013C08F010E5F1F4FFE01C49180E28C0F00
:10314000883060F4C7708D2D01C0880FCA95EAF7EA
:103150000E94431B0E946E1BE80125C08C2F0E9419
:103160004011FACF9F012E5F3F4FFE01C491CC2347
:1031700069F08FE99FE00197F1F700C00000C150AE
:10318000F6CF9F012E5F3F4FFE01F490E9010BC087
:103190000E94271BE82E07C00E943A1B0E946E1B4C
:1031A00002C00E94D5108F2D882341F0EFE9FFE087
:1031B0003197F1F700C000008150F6CFFE017ACFC1
:1031C000DF91CF911F910F91FF90EF90DF900895C5
:1031D0006093FF01709300028093010290930202BA
:1031E0000C94EF1B08956093030270930402809384
:1031F0000502909306020C94EE1B0F931F9300910F
:103200000302109104022091050230910602602B06
:10321000712B822B932B6093030270930402809393
:103220000502909306021F910F910C94EE1B0F93D1
:103230001F93009103021091040220910502309126
:103240000602602371238223932360930302709309
:10325000040280930502909306021F910F910C9433
:10326000EE1B0F931F930091030210910402209113
:103270000502309106026027712782279327609309
:1032800003027093040280930502909306021F913B
:103290000F910C94EE1B60E070E0CB010C94E818E9
:1032A0000F931F9341E050E060E070E08A019B01C2
:1032B00004C0000F111F221F331F8A95D2F7C901C6
:1032C000B8011F910F910C94E8180F931F9341E0E0
:1032D00050E060E070E004C0440F551F661F771F88
:1032E0008A95D2F78091FF0190910002A09101028E
:1032F000B09102028A019B01082B192B2A2B3B2B30
:10330000C901B8011F910F910C94E8180F931F93F6
:1033100041E050E060E070E004C0440F551F661FBC
:10332000771F8A95D2F7409550956095709580915A
:10333000FF0190910002A0910102B09102028A0166
:103340009B01082319232A233B23C901B8011F919C
:103350000F910C94E8180F931F9341E050E060E048
:1033600070E004C0440F551F661F771F8A95D2F77F
:103370008091FF0190910002A0910102B0910202A0
:103380008A019B01082719272A273B27C901B80171
:103390001F910F910C94E8180F931F930091FF0158
:1033A000109100022091010230910202602B712BDA
:1033B000822B932B1F910F910C94E8180F931F935E
:1033C0000091FF0110910002209101023091020250
:1033D00060237123822393231F910F910C94E8188B
:1033E0000F931F930091FF011091000220910102A1
:1033F0003091020260277127822793271F910F9136
:103400000C94E81808958F929F92AF92BF92DF922A
:10341000EF92FF920F931F93CF93DF9300D000D0D2
:103420001F92CDB7DEB76B837C838D838A018C813D
:103430009D81892B21F01F3F29F44F3F19F480E033
:1034400090E04CC08B818823C9F18090030290905A
:103450000402A0900502B09006028091FF019091B5
:103460000002A0910102B0910202882A992AAA2A98
:10347000BB2A8FE1E82EF12CD501C4010E2C04C02B
:10348000B695A795979587950A94D2F780FF07C0C0
:10349000DE2CB8018E2D0E94281D019729F481E0B1
:1034A000E81AF10848F7D12C88E0189FF0011124A0
:1034B000E00FF11DE154FE4FD08209C088E0189F53
:1034C000F0011124E00FF11DE154FE4FD08009837B
:1034D0001A8369817A818D2D0E94281D0F900F908B
:1034E0000F900F900F90DF91CF911F910F91FF9050
:1034F000EF90DF90BF90AF909F908F900895909144
:103500000A01992321F090910B01911109C020919A
:103510000C0130910D01F90132969FEF40E030C06F
:10352000982F9695969596959F31A0F4E0910C0171
:10353000F0910D01E90FF11D877021E030E0A90144
:1035400002C0440F551F8A95E2F7CA019181892B69
:103550008183089590912C0290FF23C01F928F9336
:103560008DEA93E09F938F930E94FE050F900F903A
:103570000F900F9008959F3F39F04F5F4E3141F00B
:1035800051915813F8CF0DC05111F7CF942FF5CFAB
:103590009F3F39F0F901E90FF11D97FDFA958283FC
:1035A0000895089590910A01992321F090910B01BB
:1035B000911109C020910C0130910D01F901329651
:1035C000205E3F4F30C0982F9695969596959F31E7
:1035D000A8F4E0910C01F0910D01E90FF11D877045
:1035E00021E030E0A90102C0440F551F8A95E2F79F
:1035F000CA018095918189238183089590912C023D
:1036000090FF16C01F928F938FE893E09F938F9344
:103610000E94FE050F900F900F900F900895319625
:10362000E217F30729F090819813F9CF1082F7CFB2
:10363000089581E090E0E0910C01F0910D01E80F18
:10364000F91F1082019680329105A9F708958091A3
:103650002B02089590912B02892B80932B020895C1
:10366000809590912B02892380932B02089580935B
:103670002B02089510922B02089590912A02892B13
:1036800080932A020895809590912A02892380933D
:103690002A02089510922A020895809309020E9436
:1036A000651C909308028093070208951092090206
:1036B0001092080210920702089580910C019091D7
:1036C0000D01FC0131969C01205E3F4F80E09191FD
:1036D00091118F5FE217F307D1F70895E0910C0184
:1036E000F0910D0180912B028083E0910C01F0910B
:1036F0000D01908180912A02892B8083809109029B
:103700008823D9F10E94651C20910702309108029C
:103710008217930748F00E94651C209107023091A0
:103720000802821B930B0AC00E94651C20910702AD
:103730003091080220953095820F931F8C32914072
:1037400070F080912C0280FF08C08BEC93E09F9377
:103750008F930E94FE050F900F900E94561BE091E0
:103760000C01F0910D01908180910902892B8083D9
:103770000E945D1B81110E94561B80910C0190914B
:103780000D010C94DC0E909339018093380108955B
:103790008295982F9C7C392F36953695282F237348
:1037A00044E0249FC0011124932F982B292F2A7ABB
:1037B0002695892F8575880F822B08950895CF93BC
:1037C000DF9300D000D01F92CDB7DEB70F900F90DF
:1037D0000F900F900F90DF91CF9108950895089565
:1037E0000C945D1080914102843021F110922D02E1
:1037F00020E488E190E00FB6F894A89580936000EB
:103800000FBE2093600083B7817F846083BF83B73E
:10381000816083BF7894889583B78E7F83BF0FB60E
:10382000F894A89580916000886180936000109260
:1038300060000FBE0895CF930E9403070E943006D8
:103840000E940407C0E08C2F0E94FA06811104C078
:10385000CF5FC830C1F701C081E0CF9108950E94C9
:103860005F100C94C2141F920F920FB60F92112486
:103870008F939F93AF93BF9380912D02811113C0BB
:1038800080912E0290912F02A0913002B0913102CE
:103890004196A11DB11D80932E0290932F02A093FB
:1038A0003002B0933102BF91AF919F918F910F90F1
:1038B0000FBE0F901F90189582E084BD93E095BDD8
:1038C0009AEF97BD80936E0008952FB7F89480917A
:1038D0002E0290912F02A0913002B09131022FBFA1
:1038E00008952FB7F89460912E0270912F02809165
:1038F0003002909131022FBF0895CF92DF92EF9264
:10390000FF920F931F932FB7F89440912E0250917E
:103910002F0260913002709131022FBF6A017B014A
:10392000EE24FF248C0120E030E0C016D106E20630
:10393000F30610F4415051099A01281B390BC901B3
:103940001F910F91FF90EF90DF90CF900895CF924D
:10395000DF92EF92FF920F931F932FB7F894C090CE
:103960002E02D0902F02E0903002F09031022FBF53
:1039700097018601061B170B280B390BC616D706B5
:10398000E806F90618F0C901B80106C0C901B80176
:1039900061507109810991091F910F91FF90EF907A
:1039A000DF90CF9008951F920F920FB60F921124BF
:1039B0008F939F93AF93BF9380912E0290912F028C
:1039C000A0913002B09131020196A11DB11D8093EA
:1039D0002E0290932F02A0933002B0933102BF9138
:1039E000AF919F918F910F900FBE0F901F901895E0
:1039F0000E94E90BF8942FEF87EA91E6215080406E
:103A00009040E1F700C0000087E090EBDC0180937C
:103A10004A0290934B02A0934C02B0934D029CE05B
:103A200088E10FB6F894A895809360000FBE90933C
:103A30006000FFCF28E0929FF0011124E80FF11DF4
:103A4000E052FF4F9491892F8F7092959F70089547
:103A5000CF93C82FCB010E941A1D282F30E080E1A0
:103A6000989FA0011124422B532B4038510519F483
:103A700080E090E015C09770E92FF0E088E0C89FE3
:103A8000E00DF11D112484E0EE0FFF1F8A95E1F790
:103A9000E20FF31FEE0FFF1FE050F849859194915C
:103AA000CF91089580E090E00895089580913402C8
:103AB00080FF0BC06091110185E0689FB001112467
:103AC00075956795759567952BC081FF09C06091C5
:103AD000110185E0689FB00111247595679520C09C
:103AE00082FF07C06091110185E0689FB001112439
:103AF00017C0909135029923D1F06091100196176B
:103B000088F72091110185E0289F90011124929F50
:103B1000A001939F500D112470E0CA010E942E2530
:103B20006038710540F46115710539F002C065E037
:103B300070E0862F08958FE7089581E008958091C1
:103B4000340280FF08C060910F0170E075956795A1
:103B50007595679521C081FF06C060910F0170E0E7
:103B60007595679519C082FF04C060910F0170E0E0
:103B700010C0909135029923C1F060910E01961703
:103B8000A0F780910F01899FC001112470E00E946D
:103B90002E256038710528F46115710521F0862FF6
:103BA00008958FE7089581E0089561E070E0F4CF13
:103BB000803F21F40E94561D819504C0813F29F465
:103BC0000E94561D809338020895823F21F40E947E
:103BD000561D819504C0833F29F40E94561D809391
:103BE00037020895893F19F40E949F1D05C08A3F3E
:103BF00031F40E949F1D81958093390208958B3F77
:103C000021F40E949F1D819504C08C3F29F40E94DD
:103C10009F1D80933A020895843F21F480913602DB
:103C2000816017C0853F21F480913602826011C007
:103C3000863F21F48091360284600BC0873F21F4D7
:103C400080913602886005C0883F31F48091360249
:103C500080618093360208958D3F21F48091340273
:103C600081600BC08E3F21F480913402826005C0D8
:103C70008F3F29F480913402846080933402089548
:103C8000803F39F48091380287FF6CC0109238026F
:103C900069C0813F29F4809138021816BCF362C0D4
:103CA00090913702823F29F497FF5CC0109237024F
:103CB00059C0833F19F41916CCF354C0893F41F41D
:103CC0008091390218160CF04DC0109239024AC08A
:103CD0008A3F29F48091390287FF44C0F6CF8B3F99
:103CE00039F480913A0287FF3DC010923A023AC0FF
:103CF0008C3F29F480913A021816BCF333C0843FFC
:103D000021F4809136028E7F17C0853F21F4809187
:103D100036028D7F11C0863F21F4809136028B7F61
:103D20000BC0873F21F480913602877F05C0883F12
:103D300031F4809136028F7E8093360213C08D3F1E
:103D400021F4809134028E7F0BC08E3F21F480914C
:103D500034028D7F05C08F3F29F4809134028B7F20
:103D6000809334028091370281110EC08091380215
:103D700081110AC080913902811106C080913A02F6
:103D8000811102C010923502089580912C0283FFA8
:103D90007EC084E094E00E946505809136021F9207
:103DA0008F938FEF93E09F938F930E94FE058DEF8B
:103DB00093E00E94650580913702282F082E000CA1
:103DC000330B3F938F938AEF93E09F938F930E94DF
:103DD000FE0588EF93E00E94650580913802282F48
:103DE000082E000C330B3F938F9385EF93E09F9346
:103DF0008F930E94FE0583EF93E00E9465058091FA
:103E00003902282F082E000C330B3F938F9380EF3D
:103E100093E09F938F930E94FE058EEE93E00E94A5
:103E2000650580913A02282F082E000C330B3F9332
:103E30008F938BEE93E09F938F930E94FE0588EE05
:103E400093E00E946505809135021F928F9385EE65
:103E500093E09F938F930E94FE0583EE93E00E9470
:103E60006505809134021F928F9380EE93E09F93BB
:103E70008F930E94FE058DED93E00E9465058DB73E
:103E80009EB74C960FB6F8949EBF0FBE8DBF86E3CB
:103E900092E00E94250F0E94651C9093330280934C
:103EA000320208951F93CF93DF9380913202909155
:103EB00033020E947D1CAC0190913502992321F0C0
:103EC0002091120130E006C0209113018AE0289F62
:103ED000900111244217530708F485C080913702DE
:103EE000C0913802D091390210913A02811107C075
:103EF000C11175C0D11173C0111171C074C09F3F41
:103F000019F09F5F90933502181624F40E94561DF5
:103F1000809337028091370287FF05C00E94561DAB
:103F20008195809337021C1624F40E94561D8093BD
:103F300038028091380287FF05C00E94561D819586
:103F40008093380260913702662331F1C0913802C4
:103F5000CC2311F1062E000C770B880B990B0E94D5
:103F6000292423E333E343E35FE30E948D240E948B
:103F7000F123609337026C2FCC0F770B880B990BD2
:103F80000E94292423E333E343E35FE30E948D246B
:103F90000E94F123609338021D1624F40E949F1D95
:103FA000809339028091390287FF05C00E949F1DCE
:103FB000819580933902111624F40E949F1D8093ED
:103FC0003A0280913A0287FF05C00E949F1D8195A9
:103FD00080933A02DF91CF911F910C94C51E9F3FB1
:103FE00009F08FCF97CFDF91CF911F910895E6E32E
:103FF000F2E085E0DF011D928A95E9F71092350223
:1040000010923402089587E296E00E9465051F929F
:1040100081E08F931F9285E08F9389ED95E09F93C8
:104020008F930E94FE050F900F900F900F900F90AE
:104030000F9008958330E9F128F4813061F08230E7
:1040400009F10895853009F462C008F449C086304A
:1040500009F474C0089580911301262F30E0280FD1
:10406000311D2F3F310524F4680F6093130103C005
:104070008FEF80931301809113011F928F9382E140
:1040800095E072C080911201262F30E0280F311D7B
:104090002F3F310524F4680F6093120103C08FEFA6
:1040A00080931201809112011F928F9380E095E01E
:1040B0005BC080911101262F30E0280F311D2F3F6A
:1040C000310524F4680F6093110103C08FEF8093D2
:1040D0001101809111011F928F938DEE94E044C0E5
:1040E00080911001262F30E0280F311D2F3F310520
:1040F00024F4680F6093100103C08FEF80931001C8
:10410000809110011F928F9388ED94E02DC08091D3
:104110000F01262F30E0280F311D2F3F310524F4E9
:10412000680F60930F0103C08FEF80930F018091A0
:104130000F011F928F938FEB94E016C080910E01B8
:10414000262F30E0280F311D2F3F310524F4680F52
:1041500060930E0103C08FEF80930E0180910E01DA
:104160001F928F9384EA94E09F938F930E94FE05A1
:104170000F900F900F900F900895833081F128F4E5
:10418000813059F08230D1F00895853009F449C06A
:10419000B8F1863009F456C008958091130168176C
:1041A00020F4861B8093130102C0109213018091AA
:1041B00013011F928F9385E994E054C080911201FE
:1041C000681720F4861B8093120102C0109212011E
:1041D000809112011F928F9383E894E043C08091F5
:1041E0001101681720F4861B8093110102C0109200
:1041F0001101809111011F928F9380E794E032C0EA
:1042000080911001681720F4861B8093100102C072
:1042100010921001809110011F928F938BE594E012
:1042200021C080910F01681720F4861B80930F0135
:1042300002C010920F0180910F011F928F9382E4B0
:1042400094E010C080910E01681720F4861B8093C3
:104250000E0102C010920E0180910E011F928F93E9
:1042600087E294E09F938F930E94FE050F900F903A
:104270000F900F900895CF93C82F1F928F938CE2C9
:1042800097E09F938F930E94FE0581E090E0A0E06D
:10429000B0E0BC01CD0104C0660F771F881F991FD5
:1042A000CA95D2F70E94F3180F900F900F900F90BD
:1042B000CF910C94C214CF938732A8F58E3108F0B9
:1042C0002BC1803109F49FC0F8F4873009F464C031
:1042D000A8F4863009F024C180912C02817F8E7F62
:1042E00080932C0281E397E00E9465058BE19AE0C0
:1042F0000E94650581E080933C024CC08B30F1F157
:104300008E3009F46CC00CC1863109F4B0C020F4C1
:10431000813109F4EDC004C1893109F491C08B31B8
:1043200009F449C0FDC0883349F150F4893209F4D9
:10433000F1C0853309F4EEC0873209F0F1C0EAC05C
:10434000833409F4E7C028F48A3308F4E9C08953B8
:10435000E4C0883409F0E4C00E94C2148AE09AE004
:104360000E9465052FEF83ED90E32150804090403F
:10437000E1F700C000000E94F81C0CC088E597E03F
:104380005CC081EF99E00E94650580912C028160FC
:1043900080932C02C1E0C9C080912C02C82FC1704B
:1043A00080FFEFCF8DEF99E00E94650580912C0290
:1043B000817F8E7F3DC090912C0291FBCC27C0F96C
:1043C00081E0C827892FC0FB81F980932C02CC2380
:1043D00019F084EE99E027C086ED99E02EC0909107
:1043E0002C0292FBCC27C0F981E0C827892FC0FBA3
:1043F00082F980932C02CC2319F087EC99E013C04A
:1044000087EB99E01AC090912C0293FBCC27C0F95E
:1044100081E0C827892FC0FB83F980932C02CC232D
:1044200051F08BEA99E00E94650580912C02816031
:1044300080932C027AC08EE999E00E946505AACF8C
:104440008FE899E00E94650582E699E00E94650583
:104450008BE299E00E9465058EEF98E00E94650569
:1044600084EB98E00E94650586E898E0E6CF88E74F
:1044700098E00E9465050E94D00E1F928F938EE5F2
:1044800098E09F938F930E94FE0580910A011F92EE
:104490008F9387E498E09F938F930E94FE0580910D
:1044A00077011F928F9384E398E09F938F930E94EC
:1044B000FE0580910B011F928F9381E298E09F93FC
:1044C0008F930E94FE050E94711C9F938F937F9390
:1044D0006F938AE098E09F938F930E94FE058DB7BB
:1044E0009EB746960FB6F8949EBF0FBE8DBF52CFB3
:1044F0000E94C214C0910B0181E0C827C0930B0138
:10450000CC2329F080E098E00E9465050EC085EF7D
:1045100097E093CF80E001C08D510E943B213ACFBC
:1045200083EF97E00E946505C0E08C2FCF9108953E
:1045300080E0089580E00895CF93C82F80913C02D9
:10454000813071F020F0823009F44BC042C1E0911B
:104550000C01F0910D018081823209F03CC107C04D
:10456000E0910C01F0910D018081823261F48C2F79
:104570000E949822811104C08C2F0E945B212FC0C1
:1045800081E090E02CC08C2F0E949A22811126C0DD
:10459000C431E1F070F4CB3081F0C031D1F40E942D
:1045A000032084E297E00E94650582E080933C024C
:1045B00015C0C93259F0C83361F481E397E00E9415
:1045C000650588E297E00E94650508C010923C02EC
:1045D00004C182E297E00E946505FFC081E081701E
:1045E000FEC0C43228F5CE3108F0C1C0CB30A1F1F5
:1045F000D0F4C73009F0D3C08EE18093130182E379
:10460000809312018AE08093110184E1809310016C
:1046100088E080930F0188E280930E0188EC95E09A
:104620000E946505BFC0C33149F1C431C1F0B7C0B4
:10463000CB3409F4A9C028F4C93289F0C83361F039
:10464000AEC0C13509F49EC0C23509F499C0CE345C
:1046500009F0A5C06AE09EC00E940320A3C080911B
:104660003B02882319F010923B029CC085ED95E037
:104670000E94650581E080933C02B1C08FEA95E01D
:104680000E9465058DE995E00E9465058091130102
:104690001F928F938AE995E09F938F930E94FE0566
:1046A00088E995E00E94650586E895E00E94650529
:1046B000809112011F928F9383E895E09F938F93CF
:1046C0000E94FE0581E895E00E94650582E795E07D
:1046D0000E946505809111011F928F938FE695E0EE
:1046E0009F938F930E94FE058DE695E00E946505DD
:1046F0008CE595E00E946505809110011F928F93D3
:1047000089E595E09F938F930E94FE0587E595E0EC
:104710000E94650582E495E00E94650580910F0185
:104720001F928F938FE395E09F938F930E94FE05D6
:104730008DE395E00E94650586E295E00E9465059F
:1047400080910E011F928F9383E295E09F938F9348
:104750000E94FE0581E295E00E9465058DB79EB737
:1047600048960FB6F8949EBF0FBE8DBF1BC0CE51AA
:10477000EC2FF0E0E25DFE4F808180933B0212C09F
:1047800061E003C061E006C06AE080913B020E94E4
:104790001A2008C080913B020E94BD2003C086EC15
:1047A00095E013C080913B02882369F01F928F939C
:1047B00080EC95E09F938F930E94FE050F900F90E1
:1047C0000F900F9004C08DEB95E00E94650581E08D
:1047D00006C010923C0280E002C080E000CFCF9182
:1047E00008950E94F8236894B1110C9487240895C9
:1047F0000E946C2488F09F5798F0B92F9927B751E1
:10480000B0F0E1F0660F771F881F991F1AF0BA9574
:10481000C9F714C0B13091F00E948624B1E0089528
:104820000C948624672F782F8827B85F39F0B93F1A
:10483000CCF3869577956795B395D9F73EF4909527
:104840008095709561957F4F8F4F9F4F0895E894A5
:1048500009C097FB3EF490958095709561957F4FC8
:104860008F4F9F4F9923A9F0F92F96E9BB27939576
:10487000F695879577956795B795F111F8CFFAF486
:10488000BB0F11F460FF1BC06F5F7F4F8F4F9F4FB7
:1048900016C0882311F096E911C0772321F09EE815
:1048A000872F762F05C0662371F096E8862F70E07B
:1048B00060E02AF09A95660F771F881FDAF7880F55
:1048C0009695879597F9089557FD9058440F551F71
:1048D00059F05F3F71F04795880F97FB991F61F082
:1048E0009F3F79F087950895121613061406551FF9
:1048F000F2CF4695F1DF08C0161617061806991F65
:10490000F1CF86957105610508940895E894BB2759
:1049100066277727CB0197F908950E94A0240C946D
:1049200011250E94032538F00E940A2520F09523C6
:1049300011F00C94FA240C94002511240C94872473
:104940000E94642470F3959FC1F3950F50E0551FAA
:10495000629FF001729FBB27F00DB11D639FAA27D4
:10496000F00DB11DAA1F649F6627B00DA11D661F23
:10497000829F2227B00DA11D621F739FB00DA11D44
:10498000621F839FA00D611D221F749F3327A00DFE
:10499000611D231F849F600D211D822F762F6A2F9A
:1049A00011249F5750409AF0F1F088234AF0EE0FFF
:1049B000FF1FBB1F661F771F881F91505040A9F72C
:1049C0009E3F510580F00C94FA240C9487245F3F9D
:1049D000E4F3983ED4F3869577956795B795F79568
:1049E000E7959F5FC1F7FE2B880F911D96958795E0
:1049F00097F9089597F99F6780E870E060E008955F
:104A00009FEF80EC089500240A94161617061806E6
:104A10000906089500240A941216130614060506C2
:104A20000895092E0394000C11F4882352F0BB0F53
:104A300040F4BF2B11F460FF04C06F5F7F4F8F4FB6
:104A40009F4F0895991B79E004C0991F961708F0AD
:104A5000961B881F7A95C9F78095089597FB072EB6
:104A600016F4009407D077FD09D00E94482507FC72
:104A700005D03EF4909581959F4F0895709561956E
:104A80007F4F0895EE0FFF1F0590F491E02D0994DC
:104A9000AA1BBB1B51E107C0AA1FBB1FA617B70764
:104AA00010F0A61BB70B881F991F5A95A9F7809580
:0C4AB0009095BC01CD010895F894FFCF53
:104ABC000C07FD07DA07A607720701010A0228088E
:104ACC00140A321E404D362239F702AA02740252E1
:104ADC000219028C01A501BE01D701F701000102E8
:084AEC00030405060708090098
:106800000000000000000000040005000600070072
:10681000080009000A000B000C000D000E000F001C
:1068200010001100120013001400150016001700CC
:10683000180019001A001B001C001D001E001F007C
:10684000200021002200230024002500260027002C
:106850002800000035002B002C002D002E002F00FA
:1068600030002A00000033003400290036003700D1
:106870003800E00000000000000000000000000000
:106880000000000000000000000000000000000008
:1068900000000000000000000000000000000000F8
:1068A00000000000000000000000000000000000E8
:1068B00000000000000000000000000000000000D8
:1068C00000000000000000000000000000000000C8
:1068D00000000000000000000000000000000000B8
:1068E0000000000000000000310000000000000077
:1068F0000000E100E200E300F1A1E500E600E700AE
:106900000000000000000000EA4401000100E24431
:106910000100010001005500460054004A004B00F0
:10692000560057004700480001000100E9440100FB
:106930000100010001000100010001003A003B00DC
:106940003C003D003E003F0040004100420043004B
:10695000580000004C00390001004400450052007E
:1069600001000100000050004F0081404D004E002A
:1069700051000100000000000000000000000000C5
:106980000000000000000000000000000000000007
:1069900000000000000000000000000000000000F7
:1069A00000000000000000000000000000000000E7
:1069B00000000000000000000000000000000000D7
:1069C00000000000000000000000000000000000C7
:1069D00000000000000000000000000000000000B7
:1069E000000000000000000049000000000000005E
:1069F0000000010001000100010001000100010090
:00000001FF
